:020000040000FA
:0400000068303A2802
:08000800A000030EA100831209
:1000100081018B100B11210E8300A00E200E090010
:0C007400203084008001840A80300402E7
:10008000031C3C281230B0003B2183160C30850540
:1000900087018312850187010730990000309A009B
:1000A000103083168E008312603083168F00831207
:1000B0000030831691009F008312C83083168100A0
:1000C000831231309000003083168C008312103080
:1000D0008B00831600309B001C141A088312BC008E
:1000E000851D5D213C1C7C28831610309B001C1450
:1000F0001A088312BD00472181018E018F010B1167
:100100008B100B108C018B17982031199A201D2110
:10011000B30B9628031085190314B90DF03039027A
:10012000031959210F3039020319552183218428DD
:1001300064000800080031110130B7008B13203033
:10014000370783169B001C141A088312A400103072
:10015000370783169B001C141A088312A300003073
:10016000370783169B001C141A088312A2008B17F2
:10017000321CC02822090339A200A309A409A50939
:1001800001303702031DC9283D18C9283D143E140B
:100190003C2101303702031DD2283D1CD2283D10DE
:1001A0003E143F21D328B70A023037020318080053
:1001B0009E280130B600B300B400B500B700850139
:1001C0008701B1139820B30BF52803108519031488
:1001D000B90DF030390203191329B40BF528013099
:1001E0003702031943219630B400311DE228311142
:1001F000321CFF282D090339AD00AE09AF098B135E
:1002000020303707BB002F08BA00262110303707EF
:10021000BB002E08BA00262100303707BB002D088E
:10022000BA0026218B1785018701B70AB601023073
:100230003702031CE228472108003E1C08003E103C
:100240001030BB003D08BA00262108008B133A0885
:1002500083161C159A0083123B0883169B005530A9
:100260009D00AA309D009C1464009C1834291C1128
:1002700083128B17080008000130BD0008008701B9
:100280000530D40008000508333A85000800BD0198
:100290003D14080001303D0203194F2908000130C8
:1002A000D40056150730D30008003D143E143C21FD
:1002B00008003D103E143F210800B601B301B4010F
:1002C0003C1C6529BC01BC146729BC013C143C08DA
:1002D000B60064006B296C296D296E296F293330B3
:1002E000B41B8500B41F8501B30B6929B40B6929C0
:1002F0000310B60CB608031D69290030BB003C088A
:10030000BA00262108008F08031908008E018F010A
:10031000D0080319D329D00FA02956180516D618CE
:10032000851656190514D6198514D60158180512C4
:10033000D818851258190510D8198510D801D32955
:100340005008D10056180516D618851656190514EA
:10035000D619851451080E020318BA295818051227
:10036000D818851258190510D8198510FF30500279
:10037000031908008F08031D0800982051080E0279
:10038000031CBA2956180512D618851256190510DD
:10039000D619851058180516D81885165819051439
:1003A000D8198514080000305302031DEC293D18AC
:1003B000E429051A58140130051AD000851AD814FA
:1003C0000130851AD00008000130D40056140130E5
:1003D000D0000130D3000800051AF2295614851AFE
:1003E000D814F429D61458140130D000D40B0800C6
:1003F00001305302031D062AD6150530D400023001
:10040000D3003D180800D601D30108000230530282
:10041000031D182A56158714D8150330D40003304D
:10042000D3003D1808008701D601D301D815080074
:1004300003305302031D282A871407150330D40004
:100440000430D3003D1808008701D3015815080077
:1004500004305302031D392A87140715071403308B
:10046000D4000530D3003D1808008701D30158158A
:10047000080005305302031D4B2A87140715071483
:1004800087160330D4000630D3003D1808008701DA
:10049000D3015815080006305302031D5E2A871445
:1004A00007150714871607160330D4000730D3004A
:1004B0003D1808008701D301581508000730530282
:1004C000031D722A87140715071487160716871548
:1004D0000130D4000730D3003D1808008701D30154
:0A04E000581508000030D300080092
:084000000700030004000800A2
:02400E00CC33B1
:10420000FF00FF00FF00FF00FF00FF00FF00FF00B6
:10421000FF00FF00FF00FF00FF00FF00FF00FF00A6
:104220000100FF00FF00FF00FF00FF00FF00FF0094
:10423000FF00FF00FF00FF00FF00FF00FF00FF0086
:104240001000FF00FF00FF00FF00FF00FF00FF0065
:10425000FF00FF00FF00FF00FF00FF00FF00050060
:10426000FF00FF00FF00FF00FF00FF00FF00FF0056
:10427000FF00FF00FF00FF00FF00FF00FF00FF0046
:10428000FF00FF00FF00FF00FF00FF00FF00FF0036
:10429000FF00FF00FF00FF00FF00FF00FF00FF0026
:1042A000FF00FF00FF00FF00FF00FF00FF00FF0016
:1042B000FF00FF00FF00FF00FF00FF00FF00FF0006
:1042C000FF00FF00FF00FF00FF00FF00FF00FF00F6
:1042D000FF00FF00FF00FF00FF00FF00FF00FF00E6
:1042E000FF00FF00FF00FF00FF00FF00FF00FF00D6
:1042F000FF00FF00FF00FF00FF00FF00FF000000C5
:00000001FF
